:10000E00323032322D30372D3132202D20313233F5
:05001E00343536370007
:10174D007BFF7A00790E7D2D120026EA494B601F32
:10175D007BFF7A00790E7D2D120026E92402F9E433
:10176D003AFA900DD3EBF0A3EAF0A3E9F08004E48C
:10177D00FEFF22900DD3E0FBA3E0FAA3E0F9900069
:10178D0001120FC0FF3395E0FEC3EF9430EE64807D
:10179D0094804016D3EF9439EE64809480500B9072
:1017AD000001120FC024D0FF802E900001120FC037
:1017BD00FF3395E0FEC3EF9461EE64809480401694
:1017CD00D3EF9466EE64809480500B900001120F5D
:1017DD00C024A9FF80027F00EF7D00FC120FA7FF40
:1017ED003395E0FEC3EF9430EE64809480401ED3B9
:1017FD00EF9439EE648094805013900DD3E0FBA3E9
:10180D00E0FAA3E0F9120FA724D0FF8033900DD397
:10181D00E0FBA3E0FAA3E0F9120FA7FF3395E0FE7A
:10182D00C3EF9461EE648094804013D3EF9466EE21
:10183D00648094805008120FA724A9FF80027F00B6
:10184D00EFC454F04CFC900DD3E0FBA3E0FAA3E001
:10185D00F9900002120FC0FF3395E0FEC3EF9430F4
:10186D00EE648094804016D3EF9439EE64809480BA
:10187D00500B900002120FC024D0FF8039900DD371
:10188D00E0FBA3E0FAA3E0F9900002120FC0FF33D2
:10189D0095E0FEC3EF9461EE648094804016D3EF23
:1018AD009466EE64809480500B900002120FC02459
:1018BD00A9FF80027F00EF75F010A4FFE5F04CFE4C
:1018CD00EF4DFF900DD3E0FBA3E0FAA3E0F99000FC
:1018DD0003120FC0FD3395E0FCC3ED9430EC648032
:1018ED0094804016D3ED9439EC64809480500B9025
:1018FD000003120FC024D0FD8039900DD3E0FBA35F
:10190D00E0FAA3E0F9900003120FC0FD3395E0FC5F
:10191D00C3ED9461EC648094804016D3ED9466EC35
:10192D0064809480500B900003120FC024A9FD8099
:06193D00027D00EF4DFFEA
:011943002281
:1013F600E47880F61238F6C2B575840F75E104E418
:10140600F5E275E344F58475B7B075840F758A8384
:10141600F597438901758D01758F01758E04900DC1
:10142600D1F0A3F0900DD2E004F07006900DD1E05B
:1014360004F0900DD1E07004A3E0640F70E64389D8
:1014460002E4900DD1F0A3F0900DD1E0FEA3E0FFF1
:10145600E4FCFD7B507AC3F9F8D31212114016E56D
:101466008954107010900DD2E004F070DB900DD10D
:10147600E004F080D3759702123864E4FF123883D3
:1014860043EF04E4900DD1F0A3F0900DD1E0FEA35C
:10149600E0FFC39402EE940050157D0112370090D0
:1014A6000DD2E004F070E3900DD1E004F080DBE4AF
:1014B600F520C20AC208C20EC20DC20CD20F788035
:1014C600F608F67826F618F6782CF6900DD1F0A3E5
:1014D600F0900DD1E0FEA3E0FFC3EE9401501C7422
:1014E600192FF582740C3EF583E4F0900DD2E004DA
:1014F600F070DE900DD1E004F080D6E4900DD1F0CE
:10150600A3F0900DD1E0FEA3E0FFC39440EE94005B
:10151600501C74192FF582740D3EF583E4F0900D7E
:10152600D2E004F070DC900DD1E004F080D41239E2
:1015360029E4F584E5EF54027010E5EF5408D394DE
:1015460000748094804003D38001C392037D08E435
:10155600FF123316E4782BF67823F6900DB4E0FBF1
:10156600A3E0FAA3E0F97823E6FF75F010A4F5826C
:1015760085F083120FC0FE782B26F6EE60057823E1
:101586000680D8D3EF9400748094804035900DB4D3
:10159600E0FBA3E0FAA3E0F990000D1212BB120FD4
:1015A600A7FF7455120FED120FA764556002D20CF7
:1015B60074AA120FED120FA764AA6002D20CEF12E2
:1015C6000FEDE4F584E5EF5402D394007480948023
:1015D60040047F018002E4FF1220CD900DD0EFF091
:1015E600900DD0E05401703CC20974FF782EF608C5
:1015F600F608F608F67E007F107D007B007A0079FB
:1016060034121342900DD674FFF0A37419F0A3742C
:1016160044F0A3E4F0A37410F07B007A007934124E
:1016260031F48002D20912174D7832A60608A607B1
:10163600900DD0E054026003021715A3F0A3F090BA
:101646000DD2E0C4F8540FC868FF900DD1E0C45421
:10165600F048FE900DB4E0FBA3E0FAA3E0F98F8218
:101666008E83120FC0700302170CE92FF9EA3EFAB7
:10167600900004120FC020E27CE4900DCFF0900D94
:10168600CFE0FDC3784796506C900DD2E0C4F85475
:101696000FC868FF900DD1E0C454F048FE900DB419
:1016A600E0FBA3E0FAA3E0F98F828E83120FC0FF5E
:1016B6007E00C006C0077C00900DD2E0C4F8540F2F
:1016C600C868FF900DD1E0C454F048FEE92FF9EA4E
:1016D6003EFA90000D1212BB782BE68DF0A429F984
:1016E600EA35F0FA7D00D007D006121342900DCFEE
:1016F600E004F08089900DD2E004F07006900DD1E0
:10170600E004F00216457F0112325CC20B8007E44A
:10171600FF12325CD20BE4900DD1F0A3F0900DD104
:10172600E0FEA3E0FFC39402EE940050197A007B1A
:10173600967D0312295A900DD2E004F070DF900DC9
:06174600D1E004F080D7A1
:01174C00227A
:05392400782CE6FF22F3
:06391800EF24FF920F22D4
:06391E00A20FE433FF22BA
:03002300021B0DB0
:101B0D00C0E0C0F0C083C082C0D075D000C000C09E
:101B1D0001C002C003C004C005C006C00720990360
:101B2D00021BB8C2997826067926E7788166703A45
:041B3D00F67826F61A
:101B4100900DB7740AF0900DB7E0D39400748094AF
:101B510080401FA37413F0900DB8E0D394007480FB
:101B61009480400600E014F080ED900DB7E014F091
:021B710080D41E
:041B7300C2B5804136
:101B7700900DB77414F0900DB7E0D394007480946F
:101B870080401FA37413F0900DB8E0D394007480C5
:101B97009480400600E014F080ED900DB7E014F05B
:021BA70080D4E8
:101BA9007826E62419F582E4340DF583E0F59920C9
:101BB9009803021C85209A08200A05C298021C81F4
:101BC900C29A7825E6062419F582E4340CF583E5F2
:101BD90099F0C298E6FF7E0064017013900C19E039
:101BE900FD7004F6021C85ED54072402782DF6EFEA
:101BF90064024E700E782DE664097007900C1AE0A5
:101C09002403F67825E6FFFD7C00B40007ECB40157
:101C190003F68068EFC3782D964061ED24FFFDEC53
:101C290034FFFC7B017A0C7919122AC17825E62444
:101C390018F582E4340CF583E06F60047600803C8B
:101C4900900DB77414F0900DB7E0D394007480949C
:101C590080401FA37413F0900DB8E0D394007480F2
:101C69009480400600E014F080ED900DB7E014F088
:021C790080D415
:101C7B00782A061200A678257600D007D006D00564
:101C8B00D004D003D002D001D000D0D0D082D083EA
:051C9B00D0F0D0E032A2
:05392900782AE6FF22F0
:1027E500900C1AE075F010A4FF900DB4E0FBA3E087
:1027F500FAA3E02FF9EA35F0FA90000D1212BB901A
:102805000DBB782CE6FF18E68FF0A4FFE02FF582CC
:0F281500E435F0F583120FC0FF7B017A0D79B91E
:10282400900DC9EFF0A3EBF0A3EAF0A3E9F0E4F50F
:1028340084EA494B6028900DCAE0FBA3E0FAA3E0C8
:10284400F9120FA7FF900DC9E0FD7C001239099021
:0E2854000DCAE0FBA3E0FAA3E0F9EF120FEDCE
:10286200900DCD7414F0900DCDE0D394007480944B
:1028720080401FA37413F0900DCEE0D394007480B7
:102882009480400600E014F080ED900DCDE014F04D
:0228920080D4F0
:10289400900DC9E0F5997F0112373A3099FDC2993C
:0128A4002211
:102F0700900D197478F07825E62418F582E4340CCE
:092F1700F583E0900D1AF07F0231
:102F200090FFFF121311EFF090FFFE121311E4F562
:0F2F300084850883850982A3A3E07881F6D2B552
:102F3F008508838509827414F0850883850982E0EA
:102F4F00D3940074809480402DA37413F08508836C
:102F5F00850982A3E0D3940074809480400D00858E
:102F6F000883850982A3E014F080E2850883850930
:062F7F0082E014F080C3A3
:0C2F8500900D19E0F59990000302131163
:10341200C9EFC9E964017028EDC39B403F7847E6D4
:10342200FFEB2FFFE433FEEDC39FEE6480F8748060
:10343200985029D20AC3ED9B782CF6782776012280
:10344200CFE9CFEF6402701ACFEBCFCEEDCEEE6FA5
:10345200700AD20A782CF67827760222C20AE47819
:0334620027F62228
:102DEF00900DC9ECF0A3EDF0C9EFC9BAFF19BBFF05
:102DFF0016900DC9E06A7003A3E06B7068D20A7871
:102E0F002CF67827E9F622E964017035C3900DCAD4
:102E1F00E09B900DC9E09A40267847E62BFFE43AF5
:102E2F00FEE0FCA3E0FDC39FEC9E5013D20ACFEB54
:102E3F00CFCEEDCEC3EE9F782CF678277601228089
:102E4F0024CFE9CFEF64027022CEEACECFEBCF9042
:102E5F000DC9E06E7003A3E06F700AD20A782CF6EA
:0C2E6F007827760222C20AE47827F622B7
:1000A600900C19E0FE54F8900DBAF0E4F584EE12C7
:1000B60012EB00F50901020A011510011E11012FAC
:1000C60012014619015C1A018120018A280244297D
:1000D60003AB3303EC37042C39044641045149047D
:1000E6005C5004B06103757004A898000004E090A9
:1000F6000C1AE0FD782FE6FB7F018027900C1AE0B2
:10010600FCA3E0FD782EE6FA08E6FB7F01802BD201
:100116000A782776030204E0900C1AE0FD7831E6AF
:10012600FB7F021234120204E0900C1AE0FCA3E0FA
:10013600FD7830E6FA08E6FB7F02122DEF0204E0B6
:10014600900C1AE0FD782FE6FB7F01123412200A8C
:10015600030204E0801A900C1AE0FCA3E0FD782E5E
:10016600E6FA08E6FB7F01122DEF200A030204E0FF
:10017600900D197478F07F010204DDE4F58475EFC3
:10018600100204E0C2ACE4900DB9F0D2B57B017A5E
:100196000D79B97F7F1228247B017A0D79B97F18F2
:1001A6001228247B017A0D79B97F05122824782339
:1001B600E612281D782EE612281D782FE612281D35
:1001C6007830E612281D7831E612281D7832E612BC
:1001D600281D7833E612281DE4900DBBF0900DBB68
:1001E600E0FFC3941074809480501074342FF8E6A6
:1001F60012281D900DBBE004F080E2900DB9E0FFDF
:090206007B007A00790012282423
:10020F00900DC7740AF0900DC7E0D39400748094DA
:10021F0080401FA37413F0900DC8E0D39400748036
:10022F009480400600E014F080ED900DC7E014F0CC
:02023F0080D469
:10024100020360900C1AE0FFC37823964003020377
:1002510067EF75F010A4FF900DB4E0FBA3E0FAA3E3
:10026100E02FF9EA35F0FA900DC4EBF0A3EAF0A320
:10027100E9F0C2ACE4900DB9F0D2B57B017A0D7909
:10028100B97F7F1228247B017A0D79B97F0D12285D
:1002910024900DC4E0FBA3E0FAA3E0F9120FA7122A
:1002A100281D900DC4E0FBA3E0FAA3E0F990000142
:1002B10012281A900DC4E0FBA3E0FAA3E0F9900024
:1002C1000212281A900DC4E0FBA3E0FAA3E0F99012
:1002D100000312281A900DC4E0FBA3E0FAA3E0F991
:1002E10090000412281AE4900DBBF0900DBBE0FFC2
:1002F100C39408748094805026900DC4E0FBA3E061
:10030100FAA3E02405F9E43AFA7E00E92FF9EE3A7E
:10031100FA120FA712281D900DBBE004F080CC90BB
:0D0321000DB9E0FF7B007A0079001228245E
:10032E00900DC7740AF0900DC7E0D39400748094BA
:10033E0080401FA37413F0900DC8E0D39400748016
:10034E009480400600E014F080ED900DC7E014F0AC
:02035E0080D449
:10036000C2B5D2AC0204E0900D197478F0E4A3F0A9
:100370007F020204DD1238E3780A121272900D191E
:10038000747CF0780AE6A3F008E6A3F008E6A3F090
:1003900008E6A3F07C007D057B017A0D7919122A0D
:1003A000C1900D1EEFF07F060204DD900C1AE0FFF5
:1003B0007E006401700FA3E0FDA3E0782ECDF60867
:1003C000EDF60204A8EF64024E700A900C1BE07870
:1003D0002EF60204A8900C1AE06403700CA3E0FF50
:1003E000A3E07830CFF608EFF60204A8E4900DBB46
:1003F000F0900DBBE0FFC394107480948050279060
:100400000C1AE0FEEFC39E501D900DBBE0241BF5BF
:1004100082E4340CF583E0FE74342FF8EEF6900D90
:10042000BBE004F080CBE47843F6807C7A007B323A
:100430007D01782CE6FF12295A900C1AE0FDE4FFAA
:100440001233160204E0900C1AE024FF9202020418
:10045000E0900C1AE024FF92010204E0782CE660A0
:1004600008900DBD7402F0800E900DBD200D057436
:1004700003F080037401F0900D197479F0900DBDB4
:10048000E0900D1AF07C007D027B017A0D79191243
:100490002AC1900D1BEFF07F03122F20900DBDE0BD
:1004A0006401703CD20E8002D208788076F18030F0
:1004B0007A007B327D017F0012295A900D197479E0
:1004C000F0900C1AE0900D1AF07C007D027B017A0E
:1004D0000D7919122AC1900D1BEFF07F03122F2006
:1004E000900DBAE064A060030207BF7847E664019C
:1004F000700D300F0AFA7B327D017F0112295A906C
:100500000C19E064A16003020650A3E0C3782396AF
:100510004003020645900DB4E0FBA3E0FAA3E0F926
:10052000900C1AE0FF75F010A4F58285F083120F8D
:10053000C0900DBDF0EF75F010A4FFE92FF9EA357A
:10054000F0FA900004120FC030E23C900C1AE0FF69
:10055000120003900DBDEFF0900D19747FF0A3EF22
:10056000F02402FDE433FC7B017A0D7919122AC1D3
:10057000900DBDE0FE241BF582E4340DF583EFF011
:10058000EE2403FF0207BC900C1AE0FF120003C226
:10059000ACE4900DB9F0D2B5900DBDE0D3940674E3
:1005A00080948040377B017A0D79B97F7F122824AF
:1005B000900DBDE012281DE4900DBBF0900DBDE044
:1005C000FF900DBBE0C39F500B1227E5900DBBE0E1
:1005D00004F080E8900DBDE004F08026900DBDE0B1
:1005E000247812281DE4900DBBF0900DBDE0FF9023
:1005F0000DBBE0C39F500B1227E5900DBBE004F04C
:1006000080E8900DB9E0FF7B007A00790012282481
:10061000900DC7740AF0900DC7E0D39400748094D5
:1006200080401FA37413F0900DC8E0D39400748031
:100630009480400600E014F080ED900DC7E014F0C7
:0206400080D464
:100642000207AE900D197478F07F010207BC900C7E
:1006520019E064A260030207BF7823E6FFA3E0FE6D
:10066200C39F40030207B4A3E0FDC39F40030207F8
:10067200B4EE9D40030207B4900C1AE0900DBBF05B
:10068200E4900DC2F0A3F0900C1BE0FE900DBBE0D5
:10069200FFD39E5034120003900DB4E0FBA3E0FAA6
:1006A200A3E0F9900DBBE075F010A4F58285F0830C
:1006B200120FC0FF900DC3E02FF0900DC2E0340086
:1006C200F0900DBBE004F080BEC2ACE4900DB9F036
:1006D200D2B57B017A0D79B97F7F122824900DC2A1
:1006E200E0FEA3E0FFC39480EE94005002800F90DE
:1006F2000DC2E0448012281D900DC2A3E0FF122813
:100702001E900C1AE0900DBBF0900C1BE0FF900DB8
:10071200BBE0D39F5056E4A3F0900DB4E0FBA3E0FE
:10072200FAA3E0F9900DBBE0FF75F010A4F5828505
:10073200F083120FC0FE900DBCE0C39E5026EF75F1
:10074200F010A4FF900DB4A3A3E02FF9EA35F0FA5C
:1007520090000D1212BB900DBC122807900DBCE048
:1007620004F080B5900DBBE004F0809D900DB9E0DF
:0A077200FF7B007A007900122824B2
:10077C00900DC7740AF0900DC7E0D3940074809468
:10078C0080401FA37413F0900DC8E0D394007480C4
:10079C009480400600E014F080ED900DC7E014F05A
:0207AC0080D4F7
:1007AE00C2B5D2AC800B900D197478F07F01122F68
:1007BE0020900DBAE064587057FA7B327D01782C88
:1007CE00E6FF12295A900DCC7401F0A3740DF0A31C
:1007DE00741AF07B017A0C791A123509900DBDEF5F
:1007EE00F0E0FE2478900D19F0EE2401FDE433FCC8
:1007FE007B017A0D7919122AC1900DBDE0FE241AE3
:10080E00F582E4340DF583EFF0EE2402FF122F2073
:10081E00900DBAE0FF64806008EF64886003020AFE
:10082E002C300F367827E66401700EFA7B327D018C
:10083E00782CE6FF12295A8021E4900DBBF0900D22
:10084E00BBE0FFC378479650117A007B327D0112D0
:10085E00295A900DBBE004F080E4900C19E0540787
:10086E00900DBDF064077012900DBC04F0900C1A40
:10087E00E0900DBDF0900C1B8008E4900DBCF09044
:10088E000C1AE0900DBEF0900DBDE014F0A3E0FF49
:10089E00C37823964003020A2C900DB4E0FBA3E02C
:1008AE00FAA3E0F975F010EFA4F58285F083120F2C
:1008BE00C0FF900DBDE0D39F4002EFF07827E664B5
:1008CE0001700D782CE6900DC1F0900DC0F0800BEC
:1008DE00E4900DC0F07847E614A3F0900DC0E078D8
:1008EE002CF6900DC1E0FF782CE6D39F4003020A50
:1008FE001AE4900DBBF0900DBDE0FF900DBBE0C370
:10090E009F4003020A0C900DBEE075F010A4FF90FC
:10091E000DB4E0FBA3E0FAA3E02FF9EA35F0FA906C
:10092E000004120FC030E203020A03900001120FFE
:10093E00C064387053900DBDE0D3940474809480DD
:10094E00900DBBE0FF4010A3E02F241BF582E43492
:10095E000CF583E0FD807E7825E6C39FFFE49400CE
:10096E00FE74172FF582740C3EF583E0FD900DBEDC
:10097E00E075F010A4FF900DB4E0FBA3E0FAA3E045
:10098E002FF9EA35F0FA804D900DB4E0FBA3E0FAB2
:10099E00A3E0F9900DBEE075F010A4F58285F0830A
:1009AE00120FC0FF7825E6C39FFFE49400FE900D62
:1009BE00BBE07C002FFFEC3EFE74182FF582740C0A
:1009CE003EF583E0FD900DBEE075F010A4FFE92F1B
:1009DE00F9EA35F0FA90000D1212BB782CE6FF18EA
:1009EE00E68FF0A4FF900DBBE02FF582E435F0F515
:1009FE0083ED120FFF900DBBE004F0020904900D81
:100A0E00BEE0FF1237CD782C060208F0900DC0E044
:100A1E00782CF6900DBAE064887003122F07900DB3
:100A2E00BAE064A86003020BD0300F367827E66474
:100A3E0001700EFA7B327D01782CE6FF12295A8066
:100A4E0021E4900DBBF0900DBBE0FFC378479650AC
:100A5E00117A007B327D0112295A900DBBE004F011
:100A6E0080E4900C1AE030E718547FFEA3E0FDED11
:100A7E00FF900DC2EEF0A3EFF0900DBC7403F0806A
:100A8E0013900C1AE0FF900DC2E4F0A3EFF0900D5E
:100A9E00BC7402F0900DBCE0FF2419F582E4340C16
:100AAE00F583E0FE741A2FF582E4340CF583E090A2
:100ABE000DBFF0CFEECF900DBEEFF0900DBFE0FF6B
:100ACE00900DBEE0FED39F4003020BCDEEC3782304
:100ADE00964003020BC4900DB4E0FBA3E0FAA3E032
:100AEE00F975F010EEA4F58285F083120FC0900D0B
:100AFE00BDF07827E66401700D782CE6900DC1F0FC
:100B0E00900DC0F0800BE4900DC0F07847E614A372
:100B1E00F0900DC0E0782CF6900DC1E0FF782CE639
:100B2E00D39F4003020BB2E4900DBBF0900DBDE0DD
:100B3E00FF900DBBE0C39F505D900DBEE075F010B1
:100B4E00A4FF900DB4E0FBA3E0FAA3E02FF9EA3581
:100B5E00F0FA900004120FC020E233900DBBE0FFBC
:100B6E00A3E02F241BF582E4340CF583E0FD900006
:100B7E000D1212BB782CE6FF18E68FF0A4FF900D35
:100B8E00BBE02FF582E435F0F583ED120FFF900DEB
:100B9E00BBE004F08096900DBEE0FF1237CD782CAE
:100BAE0006020B26900DC0E0782CF6900DBDE0FFEE
:100BBE00900DBCE02FF0900DBEE004F0020AC912B9
:020BCE002F07EF
:010BD0002202
:107000007880E664F16003027B817819F608F678EF
:0470100081E6604372
:10701400900DE9740AF0900DE9E0D3940074809423
:1070240080401FA37413F0900DEAE0D394007480A1
:107034009480400600E014F080ED900DE9E014F037
:0270440080D4F6
:10704600781A06E6187001067819B627BC08B61035
:10705600B8C2AF7584015398FCE47815F618F6E4C7
:10706600F584209855E47819F608F6209848C378F0
:0A7076001AE6948818E69413503CC3
:10708000900DE9740AF0900DE9E0D39400748094B7
:1070900080401FA37413F0900DEAE0D39400748035
:1070A0009480400600E014F080ED900DE9E014F0CB
:0270B00080D48A
:1070B200781A06E61870B80680B5B2B480A87814BB
:1070C200A699C298E6FF641A6008EF640A60030298
:1070D2007267E47819F608F6209848C3781AE6949D
:0770E2008818E69413503CEE
:1070E900900DE9740AF0900DE9E0D394007480944E
:1070F90080401FA37413F0900DEAE0D394007480CC
:107109009480400600E014F080ED900DE9E014F061
:0271190080D420
:10711B00781A06E61870B80680B5209803027065D9
:10712B007815A699C298E47819F608F6209848C302
:0B713B00781AE6948818E69413503C84
:10714600900DE9740AF0900DE9E0D39400748094F0
:1071560080401FA37413F0900DEAE0D3940074806E
:107166009480400600E014F080ED900DE9E014F004
:0271760080D4C3
:10717800781A06E61870B80680B52098030270657C
:107188007815A699C298E47819F608F6209848C3A5
:0B719800781AE6948818E69413503C27
:1071A300900DE9740AF0900DE9E0D3940074809493
:1071B30080401FA37413F0900DEAE0D39400748011
:1071C3009480400600E014F080ED900DE9E014F0A7
:0271D30080D466
:1071D500781A06E61870B80680B52098030270651F
:1071E5007815A699C29818E6641A6003027B72D2D4
:0371F500B5C29987
:1071F800900DE97414F0900DE9E0D3940074809434
:1072080080401FA37413F0900DEAE0D394007480BB
:107218009480400600E014F080ED900DE9E014F051
:0272280080D410
:06722A007599783099FD12
:10723000900DE9740AF0900DE9E0D3940074809405
:1072400080401FA37413F0900DEAE0D39400748083
:107250009480400600E014F080ED900DE9E014F019
:0272600080D4D8
:10726200C2B5027B727814E6FF7E006450600302AE
:1072720073B77819F608F6209848C3781AE6948806
:0672820018E69413503CD5
:10728800900DE9740AF0900DE9E0D39400748094AD
:1072980080401FA37413F0900DEAE0D3940074802B
:1072A8009480400600E014F080ED900DE9E014F0C1
:0272B80080D480
:1072BA00781A06E61870B80680B520980302706539
:0A72CA007815A699C298D2B5C299B2
:1072D400900DE97414F0900DE9E0D3940074809457
:1072E40080401FA37413F0900DEAE0D394007480DF
:1072F4009480400600E014F080ED900DE9E014F075
:0273040080D433
:087306007599793099FDC299D7
:10730E00900DE97414F0900DE9E0D394007480941C
:10731E0080401FA37413F0900DEAE0D394007480A4
:10732E009480400600E014F080ED900DE9E014F03A
:02733E0080D4F9
:087340007599013099FDC29915
:10734800900DE97414F0900DE9E0D39400748094E2
:1073580080401FA37413F0900DEAE0D3940074806A
:107368009480400600E014F080ED900DE9E014F000
:0273780080D4BF
:06737A00E4F5993099FDD5
:10738000900DE9740AF0900DE9E0D39400748094B4
:1073900080401FA37413F0900DEAE0D39400748032
:1073A0009480400600E014F080ED900DE9E014F0C8
:0273B00080D487
:1073B200C2B5027B72EF64014E600302746DD2B5F6
:0273C200C2996E
:1073C400900DE97414F0900DE9E0D3940074809466
:1073D40080401FA37413F0900DEAE0D394007480EE
:1073E4009480400600E014F080ED900DE9E014F084
:0273F40080D443
:0873F6007599783099FDC299E8
:1073FE00900DE97414F0900DE9E0D394007480942C
:10740E0080401FA37413F0900DEAE0D394007480B3
:10741E009480400600E014F080ED900DE9E014F049
:02742E0080D408
:06743000E4F5993099FD1E
:10743600900DE9740AF0900DE9E0D39400748094FD
:1074460080401FA37413F0900DEAE0D3940074807B
:107456009480400600E014F080ED900DE9E014F011
:0274660080D4D0
:10746800C2B5027B727814E6640260030275CF78B5
:1074780019F608F6209848C3781AE6948818E6940E
:0374880013503C62
:10748B00900DE9740AF0900DE9E0D39400748094A8
:10749B0080401FA37413F0900DEAE0D39400748026
:1074AB009480400600E014F080ED900DE9E014F0BC
:0274BB0080D47B
:1074BD00781A06E61870B80680B520980302706534
:1074CD007815A699C298E408F618E6FF13B392B49E
:1074DD00EF25E0FECC7470CCCD7400CDC3E49DEEF1
:1074ED009C5029E6FD7F0025E0FEC394E0501DED84
:1074FD0020E020E4F58443B701758F03781BEEF689
:10750D0008EFF6F5828E83F0F58F8004781676FFFE
:07751D00E4F584D2B5C29928
:10752400900DE97414F0900DE9E0D3940074809404
:1075340080401FA37413F0900DEAE0D3940074808C
:107544009480400600E014F080ED900DE9E014F022
:0275540080D4E1
:087556007599783099FDC29986
:10755E00900DE97414F0900DE9E0D39400748094CA
:10756E0080401FA37413F0900DEAE0D39400748052
:10757E009480400600E014F080ED900DE9E014F0E8
:02758E0080D4A7
:087590007816E6F5993099FD2B
:10759800900DE9740AF0900DE9E0D394007480949A
:1075A80080401FA37413F0900DEAE0D39400748018
:1075B8009480400600E014F080ED900DE9E014F0AE
:0275C80080D46D
:1075CA00C2B5027B727814E6640360030277DC7842
:1075DA0019F608F6209848C3781AE6948818E694AB
:0375EA0013503CFF
:1075ED00900DE9740AF0900DE9E0D3940074809445
:1075FD0080401FA37413F0900DEAE0D394007480C3
:10760D009480400600E014F080ED900DE9E014F058
:02761D0080D417
:10761F00781A06E61870B80680B5209803027065D0
:10762F007815A699C298E47819F608F6209848C3F9
:0B763F00781AE6948818E69413503C7B
:10764A00900DE9740AF0900DE9E0D39400748094E7
:10765A0080401FA37413F0900DEAE0D39400748065
:10766A009480400600E014F080ED900DE9E014F0FB
:02767A0080D4BA
:10767C00781A06E61870B80680B520980302706573
:10768C007817A699C2987815E6FF1392B4EF25E007
:10769C00FECC7470CCCD7400CDC3E49DEE9C400345
:1076AC00027065E625E0FCC394E04003027065E4DB
:1076BC00F58443B701758F017817E675F020A42483
:1076CC0000FFE5F03C781BF608EFF6E4F58478183B
:1076DC00F67818E6C3942074809480503FE408F642
:1076EC0008F6209816C3781AE6948818E694135076
:1076FC000A000806E61870EA0680E7209803027074
:10770C0065781B0806E618CEE6CE70010614F582E5
:10771C008E83E599F0C29878180680B5E4F584F567
:07772C008FF584D2B5C2996C
:10773300900DE97414F0900DE9E0D39400748094F3
:1077430080401FA37413F0900DEAE0D3940074807B
:107753009480400600E014F080ED900DE9E014F011
:0277630080D4D0
:087765007599783099FDC29975
:10776D00900DE97414F0900DE9E0D39400748094B9
:10777D0080401FA37413F0900DEAE0D39400748041
:10778D009480400600E014F080ED900DE9E014F0D7
:02779D0080D496
:06779F00E4F5993099FDAC
:1077A500900DE9740AF0900DE9E0D394007480948B
:1077B50080401FA37413F0900DEAE0D39400748009
:1077C5009480400600E014F080ED900DE9E014F09F
:0277D50080D45E
:1077D700C2B5027B727814E6FD7C00640460030284
:1077E700792F7819F608F6209848C3781AE694880E
:0677F70018E69413503C5B
:1077FD00900DE9740AF0900DE9E0D3940074809433
:10780D0080401FA37413F0900DEAE0D394007480B0
:10781D009480400600E014F080ED900DE9E014F046
:02782D0080D405
:10782F00781A06E61870B80680B5209803027065BE
:10783F007815A699C298E625E0781DF608E4F67843
:10784F0016F67819F608F6781D0806E618CEE6CE75
:10785F0070010614F5828E83E493781626F6781A53
:10786F0006E618700106781AE6700418E6640270CE
:05787F00D6D2B5C2994C
:10788400900DE97414F0900DE9E0D39400748094A1
:1078940080401FA37413F0900DEAE0D39400748029
:1078A4009480400600E014F080ED900DE9E014F0BF
:0278B40080D47E
:0878B6007599783099FDC29923
:1078BE00900DE97414F0900DE9E0D3940074809467
:1078CE0080401FA37413F0900DEAE0D394007480EF
:1078DE009480400600E014F080ED900DE9E014F085
:0278EE0080D444
:0878F0007816E6F5993099FDC8
:1078F800900DE9740AF0900DE9E0D3940074809437
:1079080080401FA37413F0900DEAE0D394007480B4
:107918009480400600E014F080ED900DE9E014F04A
:0279280080D409
:10792A00C2B5027B72ED64054C6003027B6678196E
:10793A00F608F6209848C3781AE6948818E694134D
:02794A00503CAF
:10794C00900DE9740AF0900DE9E0D39400748094E2
:10795C0080401FA37413F0900DEAE0D39400748060
:10796C009480400600E014F080ED900DE9E014F0F6
:02797C0080D4B5
:10797E00781A06E61870B80680B52098030270656E
:10798E007815A699C298E47819F608F6209848C397
:0B799E00781AE6948818E69413503C19
:1079A900900DE9740AF0900DE9E0D3940074809485
:1079B90080401FA37413F0900DEAE0D39400748003
:1079C9009480400600E014F080ED900DE9E014F099
:0279D90080D458
:1079DB00781A06E61870B80680B520980302706511
:0A79EB007817A699C298D2B5C29988
:1079F500900DE97414F0900DE9E0D394007480942F
:107A050080401FA37413F0900DEAE0D394007480B6
:107A15009480400600E014F080ED900DE9E014F04C
:027A250080D40B
:087A270075997F3099FDC299A9
:107A2F00900DE97414F0900DE9E0D39400748094F4
:107A3F0080401FA37413F0900DEAE0D3940074807C
:107A4F009480400600E014F080ED900DE9E014F012
:027A5F0080D4D1
:107A61007599203099FD7815E625E0FC7817E675C3
:107A7100F020A42400FFE5F03C781DF608EFF6E4C1
:107A81007816F67818F67818E6C3942074809480F6
:047A91005061C299E5
:107A9500900DE97414F0900DE9E0D394007480948E
:107AA50080401FA37413F0900DEAE0D39400748016
:107AB5009480400600E014F080ED900DE9E014F0AC
:027AC50080D46B
:107AC700781DE6FE08E6F5828E83E493F5993099F2
:107AD700FD781D0806E618CEE6CE70010614F5827D
:0F7AE7008E83E493781626F67818068093C2995A
:107AF600900DE97414F0900DE9E0D394007480942D
:107B060080401FA37413F0900DEAE0D394007480B4
:107B16009480400600E014F080ED900DE9E014F04A
:027B260080D409
:087B28007816E6F5993099FD8D
:107B3000900DE9740AF0900DE9E0D39400748094FC
:107B400080401FA37413F0900DEAE0D3940074807A
:107B50009480400600E014F080ED900DE9E014F010
:027B600080D4CF
:107B6200C2B5800C7814E664067005F58475EF10D2
:0F7B72007814E6640760030270657880F6D2AF7E
:017B810022E1
:103114007F0012373A1235F020090B7A007B327D9A
:10312400017F0012295A300C0B7A007B1E7D017F2F
:103134000012295A300817300D147A007B327D01B1
:10314400782CE6FF12295AC208122630D209200B25
:103154000C300D09788076F1122630D20B300E0B2C
:10316400300D08C20E1238F6127000200D121238FB
:10317400D0E47B2C7A01F9F8C31212275002D20D45
:013184002228
:1037A100E4F58475EF027F64EFD394007480948014
:1037B10040031F80F31213F61239241238A2E4FFDA
:0C37C100FE1236C112311412244180F8AF
:10232D00005EBCE2613FDD83C29C7E20A3FD1F41A8
:10233D009DC3217FFCA2401E5F01E3BD3E6082DC98
:10234D00237D9FC1421CFEA0E1BF5D0380DE3C6288
:10235D00BEE0025CDF81633D7C22C09E1D43A1FF78
:10236D004618FAA427799BC584DA3866E5BB590768
:10237D00DB856739BAE406581947A5FB7826C49A58
:10238D00653BD987045AB8E6A7F91B45C6987A2448
:10239D00F8A6441A99C7257B3A6486D85B05E7B938
:1023AD008CD2306EEDB3510F4E10F2AC2F7193CD28
:1023BD00114FADF3702ECC92D38D6F31B2EC0E5018
:1023CD00AFF1134DCE90722C6D33D18F0C52B0EE08
:1023DD00326C8ED0530DEFB1F0AE4C1291CF2D73F8
:1023ED00CA947628ABF517490856B4EA6937D58BE8
:1023FD005709EBB536688AD495CB2977F4AA4816D8
:10240D00E9B7550B88D6346A2B7597C94A14F6A8C7
:10241D00742AC896154BA9F7B6E80A54D7896B35B7
:10242D00000000002B6096CBDDEE002C96CBDDE599
:04243D00EEF7FAFDBF
:1037F900C191420C0D0009420C150009420C0F0839
:0938090009420C17080901440AE8
:1038A200900DCF12128AFFFFFFFF900DCFE0FCA315
:0838B200E0FDA3E0FEA3E0FF2E
:0138BA0022EB
:102AC10090FFFE121311ECF0A3EDF090FFFD121335
:0F2AD10011EBF0A3EAF0A3E9F090FFFC12131150
:102AE000850883850982A3A3E4F08508838509828C
:102AF000F0A3F0900007121335E0FEA3E0FF850875
:102B000083850982E0FCA3E0FDC39FEE6480F8ECBE
:102B1000648098504C900004121335E0FBA3E0FA57
:102B2000A3E0F98D828C83120FC0FF85088385098D
:102B300082A3A3E06FFF900003121335EFF0900023
:102B400003121335E090232D93850883850982A312
:102B5000A3F0850883850982E475F001121057807F
:0B2B600092850883850982A3A3E0FF93
:062B6B00900009021311A5
:0E390900CEEDCEEE6F780EF6E690232D93FFF6
:01391700228D
:0300A30002309593
:10309500C0E0C0F0C083C082C0D0E8C0E0EEC0E0B0
:1030A500EFC0E0E59830E1055398FDD211E5983081
:1030B500E049900C16E02401FF900C15E03400FE69
:1030C500900C0DE06E7003A3E06F7002802A900CE7
:1030D50015E475F00112106D85F082F583E599F020
:1030E500900C15E064087004A3E06409700A900C64
:1030F500157400F0A37409F05398FED0E0FFD0E0FA
:0F310500FED0E0F8D0D0D082D083D0F0D0E0322E
:1035F000900C0FE0FEA3E0FF900C17E06E7003A3A9
:10360000E06F603230112FC211758401900C0FE40D
:1036100075F00112106D85F082F583E0F599900C3C
:103620000FE0640C7004A3E06409700A900C0F743E
:0736300008F0A37409F02269
:10346500900C0DE0FEA3E0FF900C15E06E7003A339
:10347500E06F6039900C0DE475F00112106D85F068
:1034850082F583E0781FF6900C0DE064087004A3C4
:10349500E06409700A900C0D7400F0A37409F078CB
:1034A5001FE6FEB40D037F0A22CFEECF22123114A0
:0234B50080AEE7
:0632BB0090FFFF12131149
:1032C100900C0DE0FEA3E0FF900C15E06E7003A3DF
:1032D100E06F6039900C0DE475F00112106D85F00E
:1032E10082F583E0850883850982F0900C0DE06406
:1032F100087004A3E06409700A900C0D7400F0A337
:0F3301007409F0850883850982E0FF80027FFF51
:0633100090000102131100
:0E28A500900DE4EBF0A3EAF0A3E9F0A3EDF050
:1028B3001238D0780F121272E47813F61232BBEF8B
:1028C300FD3395E0FCEDF47002ECF46046EF640A2E
:1028D3006041EFB40D18900DE4E0FBA3E0FAA3E030
:1028E300F97813E6FFF582758300E4020FFF900D7C
:1028F300E4E0FBA3E0FAA3E0F97813E606F58275BA
:102903008300EF120FFF900DE7E0FE7813E6FF6EF2
:102913007001221231141238D0ECC0E0EDC0E0EEA9
:10292300C0E0EFC0E0900DE8E0FFE4FCFDFE780FAF
:10293300121265EF2BFBEE3AFAED39F9EC38F8D0C9
:10294300E0FFD0E0FED0E0FDD0E0FCD31212274040
:06295300030228BF7F0013
:01295900225B
:10363700900C18E02401FD900C17E03400FC900C6E
:103647000FE06C7003A3E06D700122900C17E47516
:10365700F00112106D85F082F583EFF0900C17E002
:10366700640C7004A3E06409700A900C177408F0E6
:05367700A37409F0221C
:10384500900C0FE0FEA3E0FF900C17E06E7003A351
:0F385500E06F600A7F0012373A1235F080E222EE
:1035A7007E007F09900C15EEF0A3EFF0900C0DEE66
:1035B700F0A3EFF07E087F09900C17EEF0A3EFF071
:1035C700900C0FEEF0A3EFF07E087F007D007B01EB
:1035D7007A0079091213427E047F007D007B017A0D
:0935E700087909121342D21122E5
:10331600EF7025F5847598D0F584759115F584754B
:10332600C90875CBFFED90242C93F5CA75C804E443
:10333600F584D2ACC2BC8029758401759850E4F539
:1033460084E589540F4420F589758E02CFEDCFEFC1
:1033560090243693F58DD28E43E74043F7401235DD
:03336600A7D2AF3C
:013369002241
:10318500900C0912128A00000000900C1112128A8C
:10319500000000009000007464F0E4780FF6780FEA
:1031A500E6C39402748094805044E6FF25E025E050
:1031B5002401F582E43400F583E4F0EF25E025E011
:1031C5002402F582E43400F583E4F0EF25E025E000
:1031D5002403F582E43400F583E4F0EF25E025E0EF
:0E31E5002404F582E43400F583E4F00680B0A3
:0131F30022B9
:10386400D2AFD2A9C2BBE4F584E589540F4401F573
:0F38740089758E02758CAFE4F58AD28C0231858E
:06220B0090FFFF12131109
:10221100850883850982E4F0850883850982E0FFCA
:10222100C39402748094804003022327EF25E025A4
:10223100E02404F582E43400F583E0FF7C00D394CC
:10224100007480948050030222F2850883850982FC
:10225100E025E025E02402F582E43400F583E06026
:10226100030222F2EF30E00DD39401748094804098
:10227100047D0080027D01850883850982E0FF12CB
:102281002C20850883850982E0FF25E025E02404D0
:10229100F582E43400F583E0640170057D01122CC0
:1022A10020850883850982E0FF25E025E02404F5E7
:1022B10082E43400F583E014F0EF25E025E0240406
:1022C100F582E43400F583E060278508838509827F
:1022D100E0FF25E025E02403F582E43400F583E006
:1022E100FEEF25E025E02402F582E43400F583EEDB
:1022F100F0850883850982E0FF25E025E02402F5C9
:1023010082E43400F583E06011EF25E025E024024A
:10231100F582E43400F583E014F0850883850982B1
:06232100E004F0022219A5
:06232700900001021311F9
:03000B00022CBE06
:102CBE00C0E0C0F0C083C082C0D0E8C0E0E9C0E090
:102CCE00EAC0E0EBC0E0ECC0E0EDC0E0EEC0E0EF4B
:102CDE00C0E0758CAF900C09E0FCA3E0FDA3E0FE14
:102CEE00A3E02401FFE43EFEE43DFDE43CFC900C39
:102CFE000912127E900000E014F0E07025900C1185
:102D0E00E0FCA3E0FDA3E0FEA3E02401FFE43EFE11
:102D1E00E43DFDE43CFC900C1112127E9000007418
:102D2E0064F012220B123823D0E0FFD0E0FED0E088
:102D3E00FDD0E0FCD0E0FBD0E0FAD0E0F9D0E0F836
:0B2D4E00D0D0D082D083D0F0D0E03293
:1037000090FFFF121311EDF090FFFF121311EFF075
:10371000850883850982E0FFC394027480948050F9
:1037200013A3E0FEEF25E025E02401F582E4340058
:0A373000F583EEF090000202131181
:10295A0090FFFE121311EAF0A3EBF090FFFF12139F
:10296A0011EDF090FFFF121311EFF085088385092E
:10297A0082E0FFC39402748094804003022A09EF24
:10298A0025E025E02404F582E43400F583E0706F45
:10299A00850883850982E0FB25E025E02402F5828B
:1029AA00E43400F583E07057850883850982A3E043
:1029BA0025E004FF850883850982E0FA25E025E001
:1029CA002404F582E43400F583EFF0850883850951
:1029DA0082A3A3E0FEA3E0FF7C007D0A121021EA95
:1029EA0025E025E02403F582E43400F583EFF0EBDB
:1029FA0025E025E02402F582E43400F583E4F09032
:052A0A0000040213119D
:102C200090FFFF121311EDF090FFFF121311EFF060
:062C300090FFFF121311DA
:102C3600850883850982A3E0FFFD7C00C3940274A6
:102C4600809480502CEF25E025E02401F582E434C1
:102C560000F583E0601B850883850982A3A3E070E5
:102C6600047F0180027F00850883850982A3A3EF84
:102C7600F0850883850982E584F075840FED4C7034
:102C86000F850883850982A3A3E024FF92B48019E7
:102C9600850883850982A3E06401700D8508838514
:102CA6000982A3A3E024FF92B3850883850982E005
:022CB600F584A3
:062CB8009000030213115D
:1038D000C2AF900C09E0FCA3E0FDA3E0FEA3E0FF73
:0238E000D2AF65
:0138E20022C3
:1038E300C2AF900C11E0FCA3E0FDA3E0FEA3E0FF58
:0238F300D2AF52
:0138F50022B0
:10373A0090FFFF121311EFF0850883850982E0706C
:10374A00057845F608F63010167844E675F064A454
:10375A00FFC37846E69F18E695F0500375FFA590DB
:05376A00000102131133
:10388300D210E47845F608F6EF78446003F6800238
:0F389300760A75FF0775FFA5E4F58475EF04222B
:1038F600C210E47845F608F6784476FF75FFDE7563
:03390600FFAD22F0
:10382300784606E6187001063010167844E675F0FF
:1038330064A4FFC37846E69F18E695F0500375FF2E
:02384300A522BC
:0836C100900DCFEEF0A3EFF035
:1036C900E4A3F0A3F0900DCFE0FEA3E0FFC3900DBB
:1036D900D2E09F900DD1E09E501C7FE87E0312300E
:1036E900147F0112373A900DD2E004F070D7900D93
:0636F900D1E004F080CFD7
:0136FF0022A8
:08301400900DD3EEF0A3EFF0E4
:10301C00D394FAEE94005023900DD3A3E0FFEFD39A
:10302C0094007480948040607E16EED3940074807B
:10303C0094804004001E80F21F80E3900DD3E0FFCB
:10304C00A3E0A3CFF0A3EFF0D3900DD6E094FA90C9
:10305C000DD5E0940040177FFA7E00123014900DCD
:10306C00D6E02406F0900DD5E034FFF080DAD39052
:10307C000DD4E09400900DD3E09400400B900DD54E
:08308C00E0FEA3E0FF12301486
:013094002219
:102D5900900DDF7401F0A3740DF0A374D9F07B0119
:062D69007A0D79D77D020E
:0E2D6F00900DDBEBF0A3EAF0A3E9F0A3EDF08A
:102D7D007F0112373A900DDFE0FBA3E0FAA3E0F9F3
:102D8D001210832400FFE5F034E0FE900DDBE0F936
:102D9D00A3E0FAA3E0900DE2C9F0A3EAF0A3E9F0F5
:102DAD00E4FD900DDEE0FCEDC39C5022EF2DF5828D
:102DBD00E43EF583E493FC900DE2E0FBA3E0FAA37F
:102DCD00E0F98D82758300EC120FFF0D80D4900D0C
:102DDD00DEE0FFA3E0FBA3E0FAA3E0F9E48FF0024D
:022DED0010AE26
:10270D00900DEB7412F0A37434F0900DF37401F08E
:10271D00A3740DF0A374EDF07B017A0D79EB7D02BE
:0E272D00900DEFEBF0A3EAF0A3E9F0A3EDF0BE
:10273B007880E664F160030227E41238F6C2AFE456
:10274B00F58443B701758F01A3E0FBA3E0FAA3E087
:10275B00F91210832400FFE5F034E07814F608EF4B
:10276B00F6900DEFE0FBA3E0FAA3E0F97818C6EBC7
:10277B00C608C6EAC608C6E9C6E47816F6900DF296
:10278B00E0FF7816E6C39F50327818CBE6CB0808EB
:10279B0006E618CAE6CA70010614F9120FA77817D5
:1027AB00F6E6FF78140806E618CCE6CC70010614A2
:1027BB00F5828C83EFF078160680C2E4F58F900DCE
:1027CB00F2E0FFA3E0FBA3E0FAA3E0F9E48FF01241
:0927DB0010AED2AFE4FF12388306
:0127E40022D2
:1034B7007880E664F1704AC2AF1238F6E4F58443C7
:1034C700B701758F03781576E008F67814F6781447
:1034D700E6C3940874809480501E08E6FE08E6F55B
:1034E700828E83E4F07F0112373A7816E426F618C5
:1034F700740236F6180680D6E4F58FD2AFFF12387D
:013507008340
:0135080022A0
:102630001234B7E4900DEDF0A3F07B01900DF3049C
:10264000F0A3740DF0A374EDF01B7A00792E7D16C3
:1026500012272D12270DE4900DEAF0900DEAE0C349
:102660007847964003022705E4900DE9F0900DB4F9
:10267000E0FBA3E0FAA3E0F9900DE9E0FF75F010AC
:10268000A4F58285F083120FC06071EF75F010A47D
:10269000FF900DB4A3A3E02FF9EA35F0FA90000DF6
:1026A0001212BB900DEAE0FF782BE68FF0A429F917
:1026B000EA35F0FAEBC0E0EAC0E0E9C0E0900DB422
:1026C000E0FBA3E0FAA3E0F9900DE9E075F010A4B7
:1026D000F58285F083120FC0FD900DF37401F0A315
:1026E000740DF0A374EDF0D0E0F9D0E0FAD0E0FB87
:1026F00012272D900DE9E004F002266D900DEAE01E
:0C27000004F002265B12270DE47880F63E
:01270C0022AA
:0520CD00900DD3EFF0BF
:1020D200E4900DD9F0A3F0900DD6F07B01900DDFC6
:1020E20004F0A3740DF0A374D9F01B7A00792E7D4D
:1020F20016122D6F122D59900DD7E0B4120CA3E0D9
:10210200B43407900DD6E04401F0E4900DD5F09080
:102112000DD5E0C378479640030221EFE4900DD439
:10212200F0900DB4E0FBA3E0FAA3E0F9900DD4E047
:10213200FF75F010A4F58285F083120FC0700302C0
:1021420021E6900DD3E0606AEF75F010A4FF900DC8
:10215200B4A3A3E02FF9EA35F0FA90000D1212BBF6
:10216200900DD5E0FF782BE68FF0A429F9EA35F03F
:10217200FAEBC0E0EAC0E0E9C0E0900DB4E0FBA3F6
:10218200E0FAA3E0F9900DD4E075F010A4F5828591
:10219200F083120FC0FD900DDF7401F0A3740DF0F7
:1021A200A374D9F0D0E0F9D0E0FAD0E0FB122D6FA1
:1021B2008029900DB4E0FBA3E0FAA3E0F9900DD4DE
:1021C200E075F010A4F58285F083120FC0FF900D28
:1021D200DAE02FF0900DD9E03400F0900DD4E00455
:1021E200F0022123900DD5E004F0022111122D59A5
:1021F200900DD7E0B4120CA3E0B43407900DD6E0F2
:082202004402F0900DD6E0FF4C
:01220A0022B1
:101944005350444C465278780001320000004F6EE8
:10195400000000000000010D87041C00000052502C
:101964004D446D640000010D88041C0000005250B9
:101974004D4D65617300010D8C013200000041631F
:101984006B4572720000010D900436000000537420
:10199400617475730000010D910408000001544343
:1019A4006F6E76000000010D950408000001544D8F
:1019B4006F746F720000010D990406000001494D17
:1019C4006F746F720000010D9D01340000086430D3
:1019D400000000000000010DA10134000008643182
:1019E400000000000000010DA20134000008643270
:1019F400000000000000010DA3013400000864335E
:101A0400000000000000010DA4013400000864344B
:101A1400000000000000010DA50134000008643539
:101A2400000000000000010DA60134000008643627
:101A3400000000000000010DA70134000008643715
:101A4400000000000000010DA80134000008643803
:101A5400000000000000010DA901340000086439F1
:101A6400000000000000010DAA01340000086431E8
:101A7400300000000000010DAB01340000086431A7
:101A8400310000000000010DAC0134000008643195
:101A9400320000000000010DAD0134000008643183
:101AA400330000000000010DAE0134000008643171
:101AB400340000000000010DAF013400000864315F
:101AC400350000000000010DB0013400000864314D
:101AD400360000000000010DB1013400000864313B
:101AE400370000000000010DB201340000086465F5
:101AF4006D6F00000000010DB30000000000000045
:091B0400000000000000000000D8
:10381200014701430DB4FF194D440D830000000020
:10325C00EF601D900D8812128A00000000900D8CFA
:10326C0012128A00000000E4900D87F0900DB3F06C
:10327C00900D9112128A00000000E4FFEFC394102D
:10328C0074809480500F74A12FF582E4340DF58373
:10329C00E4F00F80E77D077F0112331675840F75FC
:0F32AC00A481C287E4900D59F0A3F0FF023918F6
:1037CD0090FFFF121311EFF0850883850982E0FF4A
:1037DD00C3940274809480500D74592FF582E43493
:0C37ED000DF5837401F09000010213112F
:08000300900DC9EFF07F00220F
:10350900900DC9EBF0A3EAF0A3E9F0900DC9E0FB37
:10351900A3E0FAA3E0F9120FA7FF900DCCE0FBA3FB
:10352900E0FAA3E0F9EF120FED900DC9E0FBA3E07B
:10353900FAA3E0F9900001120FC0FF900DCCE0FB57
:10354900A3E0FAA3E0F9900001EF120FFF7F022236
:06336A007B017A0D796F72
:0E337000900DE4EBF0A3EAF0A3E9F0A3EDF07A
:10337E00E4A3F0A3F0900DE7E0FFA3E0FCA3E0FDD3
:10338E00C39FEC94005026900DE4E0FBA3E0FAA35B
:10339E00E0F98D828C83120FC0FF123637900DE943
:1033AE00E004F070D0900DE8E004F080C8023845DB
:052F9100900DFEEFF0C1
:102F96001238D0900DFF12127E900C0DE0FEA3E0C9
:102FA600FF900C15E06E7003A3E06F6028900C0D87
:102FB600E475F00112106D85F082F583E0FF900C48
:102FC6000DE0B4080FA3E0B4090A900C0D7400F0EC
:102FD600A37409F0221238D0C004C005C006AB079E
:102FE600900DFEE0FFE4FCFDFEA3E0F8A3E0F9A3EC
:102FF600E0FAA3E02FFFEE3AFEED39FDEC38FCD007
:0D30060002D001D000C3121227408E7F00BF
:01301300229A
:1038BB007E007F09900C15EEF0A3EFF0900C0DEE4F
:0538CB00F0A3EFF02264
:041F8D00AD07AC06EA
:101F9100900DFD74FFF0E4900DFCF0900DFCE0FF5E
:101FA100C3941074809480501474A12FF582E4348A
:101FB1000DF583E4F0900DFCE004F080DEE4900D7B
:101FC1006FF0A3740DF0A37402F0A314F0A37410C6
:101FD100F0A37401F0E4A3F0EDA3F0ECA3F0900DF5
:101FE100F8E0FCA3E0FDA3E0FEA3E0FFE4120E6F26
:101FF1007B007AD679037848120DD27B007AFC797E
:102001007F7846120CC9120EADAC06EF900D78F038
:10201100EEA3F0900DFC740BF0900DFCE0FFC39467
:102021000F748094805014746F2FF582E4340DF591
:1020310083E4F0900DFCE004F080DEE4900DFCF010
:10204100900DFCE0FFC3940F74809480501EA3E0B8
:10205100FE746F2FF582E4340DF583E0FFC3EE9F2C
:10206100900DFDF0900DFCE004F080D4900DFDE0AA
:10207100900D7EF07D1012336A7B017A0D795B90B1
:102081000DE87464F07D101228A5EF6410900D9096
:102091007003F080037401F0E4900DFCF0900DFCEE
:1020A100E0C39410748094805021E0FF245BF5829A
:1020B100E4340DF583E0FE74A12FF582E4340DF5CF
:0B20C10083EEF0900DFCE004F080D2F4
:0120CC0022F1
:101E2300A3F07A0D79D37B01900DE27402F07F4425
:021E33007E002F
:0F1E3500900DDFEBF0A3EAF0A3E9F0AD07AC06E8
:101E4400E4900DE3F0900DE3E0FFC39412748094EA
:101E540080501474A12FF582E4340DF583E4F090DE
:101E64000DE3E004F080DEE4900D6FF0A3740BF05A
:101E7400A37402F0A314F0A3740EF0EDA3F0ECA38A
:101E8400F0E4A3F0A3F0A3F0A3F0900DE2E0900D32
:101E94007AF0E4900DE3F0900DE2E0FFA3E0FEC3DE
:101EA4009F5035900DDFE0FBA3E0FAA3E0F98E82AA
:101EB400758300120FC0FFEEFD900DE2E0C39DFD9F
:101EC400E49400FC747A2DF582740D3CF583EFF0F4
:101ED400900DE3E004F080BF7FFFE4900DE3F09009
:101EE4000DE2E0240CFDE433FCA3E0FEC39DEC64AE
:101EF40080F87480985018746F2EF582E4340DF5D0
:101F040083E0FEC3EF9EFF900DE3E004F080D090E9
:101F14000DE2E0FE247BF582E4340DF583EFF07BE3
:101F2400017A0D796FEE240DFD1233707B017A0D69
:101F3400795B900DE87464F07D071228A5EF6407BF
:101F4400900D907003F080037401F0E4900DE3F0C1
:101F5400900DE2E0240DFFE433FEA3E0C39FEE64A2
:101F640080F87480985021E0FF246FF582E4340DEA
:101F7400F583E0FE74A12FF582E4340DF583EEF0D1
:081F8400900DE3E004F080C8B9
:011F8C002232
:101CA000900DDAEEF0A3EFF0A3EBF0A3EAF0A3E9D6
:011CB000F043
:101CB100900DE074FFF07A007B327D017F011229E3
:101CC1005AE4900D6FF0A37409F0A37402F0A31409
:101CD100F0A3740DF0900DDAE0FCA3E0900D74F028
:101CE100ECA3F0E4A3F0A3F0A3F0A3F0900DE1F0D6
:101CF100900DE1E0FFC3940B74809480501E900D11
:101D0100E0E0FE746F2FF582E4340DF583E0FFC34C
:101D1100EE9F900DE0F0A3E004F080D4900DE0E0A0
:101D2100900D7AF07D0C12336A900DDFE064029021
:101D31000DE27005740AF08003740CF07B017A0DDA
:101D4100795B900DE2E0FD900DE87464F01228A536
:101D5100EF7006900D9004800F900DE2E0FEEFC34E
:101D61009E5009900D907402F07F0022E4900D9036
:101D7100F0900DE074FFF0E4A3F0900DE2E0FC14AC
:101D8100FE900DE1E0FDC39E501E900DE0E0FE745B
:101D91005B2DF582E4340DF583E0FDC3EE9D900DDE
:101DA100E0F0A3E004F080D2745A2CF582E4340D03
:101DB100F583E0FF900DE0E0FEEF6E6006900D9080
:101DC1007403F0900D61E0FFFD3395E0FCED4C6094
:101DD10005900D90EFF0E4900DE1F0900DDFE0FF44
:101DE100900DE1E0FEC39F502874622EF582E43429
:101DF1000DF583E0FF900DDCE0FBA3E0FAA3E0F931
:101E01008E82758300EF120FFF900DE1E004F080E8
:101E1100CA7A007B327D017F0012295A900DDFE0E2
:011E2100FFC1
:011E2200229D
:0E367C00900D88E0FCA3E0FDA3E0FEA3E0FFBC
:06368A00900DD512127E26
:10369000E47FE87E03FDFC900DD5E0F8A3E0F9A3FC
:1036A000E0FAA3E0FB1210E6900DD912127E7B0126
:1036B0007A0D79D9900DE27404F07F8B7E01021EA1
:0136C00035D4
:03355900EF6028F8
:10355C00900DD3E4F07406121E23900DD3E4F07496
:10356C0007121E2312367C900DD3E4F0A3740FF0D7
:06357C007B017A0D79D3FA
:10358200801F900DD1E4F0A37407F07A0D79D11267
:103592001E29900DD1E4F0A37406F07B017A0D7917
:0435A200D1121E2BF9
:0135A6002202
:10376F007B017A0D79D1900DDF7402F07F437E00DB
:10377F00121CA0EF64027019900DD2E0FE900DD1D3
:10378F00E07C002400FFEC3EFEE4FD900D91121250
:01379F007EAB
:0137A0002206
:0B2A0F00900DD1EBF0A3EAF0A3E9F07A
:102A1A007B017A0D79D4900DDF7404F07F8E7E01EC
:102A2A00121CA0EF64046003022AC0900DD7E0FFD5
:102A3A00E4FCFDFE7808121238A804A905AA06AB20
:102A4A0007900DD6E0FFE4FCFDFEEB2FFFEE3AFE09
:102A5A00ED39FDEC38FC7808121238A804A905AA49
:102A6A0006AB07900DD5E0FFE4FCFDFEEB2FFFEE71
:102A7A003AFEED39FDEC38FC7808121238A804A9A0
:102A8A0005AA06AB07900DD4E0FFE4FCFDFEEB2F90
:102A9A00FFEE3AFEED39FDEC38FCC2AFE47BE87A92
:102AAA0003F9F8121171900DD1E0FBA3E0FAA3E04B
:062ABA00F912124BD2AF2D
:012AC00022F3
:0B33BE00900DD1EBF0A3EAF0A3E9F0C2
:1033C9007B017A0D79D4900DDF7402F0121CA0EF05
:1033D90064027034900DD5E0FE900DD4E07C002499
:1033E90000FFEC3EFEC2AFAD07FCE4120E74E4FB35
:1033F900FA79207841120DD2900DD1E0FBA3E0FAC1
:08340900A3E0F912124BD2AF4F
:013411002298
:0B2B7100900DD1EBF0A3EAF0A3E9F017
:102B7C007B017A0D79D4900DDF7402F07FAF7E016A
:102B8C00121CA0EF64026003022C1F900DD5E0FE16
:102B9C00900DD4E07C002400FFEC3EFEAD07FCE47D
:102BAC00120E747B0A7AD77923783C120CC97B817C
:102BBC007A0479B5783F120DD2900DD612127EE4BC
:102BCC00FFFE7DC87C42900DD6E0F8A3E0F9A3E0AF
:102BDC00FAA3E0FB120CC9E4FBFAF9783F120BD80C
:102BEC00122540E4FBFA79C87842120DD2900DD62A
:102BFC0012127EC2AF900DD6E0FCA3E0FDA3E0FE66
:102C0C00A3E0FF900DD1E0FBA3E0FAA3E0F91212D0
:032C1C004BD2AFE9
:012C1F002292
:10244100900D59E06055E4F0900D87E0600464015F
:10245100701B900DB3E07015FA7B327D027F011283
:10246100295A12367C900D87E0FF123559900D875D
:10247100E0D394017480948040217A007B327D0204
:102481007F0112295A900D87E0FF900DCFE4F0A350
:10249100EFF07B017A0D79CF121E2B900D5AE0607F
:1024A10035E4F0900DB3E0601F900D88E0FCA3E0EF
:1024B100FDA3E0FEA3E02401FFE43EFEE43DFDE4D4
:1024C1003CFCA312127E800E7A007B327D027F01DA
:1024D10012295A12367C1238D0A804A905AA06ABD3
:1024E10007900D83E0FCA3E0FDA3E0FEA3E02464DC
:1024F100FFE43EFEE43DFDE43CFCD3121227403EE6
:10250100900DB3E070097B017A0D798C122A0F7B53
:10251100017A0D79957F297E001233BE7B017A0DF8
:1025210079997F3F7E001233BE7B017A0D799D122E
:0E2531002B7112376F1238D0900D8312127E6C
:01253F002279
:100BD100020F19E86480F8E933E83360110460F02A
:100BE100ED33EC337009E8FCE9FDEAFEEBFF22048A
:100BF10060DED3EB9FEA9EE99DE8C2E78CF0C2F785
:100C010095F0400CE8CCF8E9CDF9EACEFAEBCFFB50
:100C1100120EE485D0F05804700320D5B3E80470B7
:100C2100075002B2D5020F2392D5EC0460F7E4CC51
:100C3100C0E0C398F8603B94186008400DD0E0FB19
:100C4100020EFBE4FBFAC9FC8028E830E406E4C9A3
:100C5100FBE4CAFCE830E305E4C9CACBFCE854076D
:100C61006010F8C3E913F9EA13FAEB13FBEC13FC78
:100C7100D8F130F52FC3E49CFCEF9BFFEE9AFEED1B
:100C810099FDD0E0FBEF4E4D4C701222DB03020FB9
:100C910020EC2CFCEF33FFEE33FEED33FDED30E7BE
:100CA100EB020EFBEF2BFFEE3AFEED39FDD0E0FB40
:100CB10050130BBB0003020F23ED13FDEE13FEEFE8
:080CC10013FFEC13FC020EFB13
:100CC900EC4D6011E8497017ED33EC3304600DE425
:100CD900FCFFFEFD22E933E8330470F8020F191214
:100CE9000EE458046009E4CC248150062850090216
:100CF9000F23284003020F20C0E0EB4A7044B9805B
:100D090006D0E0FB020F0FEF4E701CBD8008EBFF11
:100D1900EAFEE9FD80EBE98DF0A4FEE5F0020DB2F3
:100D2900E9CDF9EAFEEBFFEF89F0A4FCE5F0CE8905
:100D3900F0A42EFFE435F0CD89F0A42DFEE435F0C2
:100D49008067EF4E7005BD80D780C3EF8BF0A4ACF0
:100D5900F0EE8BF0A42CFCE435F0F8EF8AF0A42C2B
:100D6900E5F038FCE433CB8DF0A42CFCE5F03BF83E
:100D7900EE8AF0A42CFCE5F038F8E433CF89F0A42E
:100D89002CFCE5F038CF3400CE89F0A42FFFE5F034
:100D99003EFEE433C98DF0A42EFEE5F039CD8AF08C
:100DA900A42FFFE5F03EFEE43DFD33D0E0FB500704
:100DB9000BBB000F020F23EC2CFCEF33FFEE33FECD
:060DC900ED33FD020EFBFC
:100DCF00020F23EC5D046005E859047003020F194C
:100DDF00120EE4580460F6EC4860F2EC7004FDFE6D
:100DEF00FF22C860DB2481C85009C39860025006F7
:100DFF00020F209850CAF582E9294B4A7005AB8241
:100E0F00020F0F75F0007C1A7880C3EF9BEE9AEDFE
:100E1F0099400DC3EF9BFFEE9AFEED99FDE842F06E
:100E2F00DC23ACF0D0E0FFD0E0FED0E0FDAB8220C1
:100E3F00E7101BEB60BAEC2CFCEF33FFEE33FEED4B
:100E4F0033FD020EFBE803F830E705C0F075F00044
:100E5F00EF2FFFEE33FEED33FD40B830E7C280AA2F
:100E6F0075F020800E75F010800575F0087D007EFE
:100E7F00007F003392D530D503121203EC334010AC
:100E8F00EF33FFEE33FEED33FDEC33FCD5F0ED2207
:0E0E9F00E5F0247EA2D513CC92E7CDCEFF2243
:100EAD00EDD2E7CD33EC3392D524814006E4FFFE3D
:100EBD00FDFC22FCE4CFCECDCC24E0501174FF809C
:100ECD00EDC3CC13CCCD13CDCE13CECF13CF047039
:070EDD00F030D5DE02120324
:10254000900DDA12127E74FFFFFEFDFC900DDAE0B2
:10255000F8A3E0F9A3E0FAA3E0FBC3121227603866
:102560007F807E967D187C4B900DDAE0F8A3E0F931
:10257000A3E0FAA3E0FB120F2E6002501B7F807EC7
:10258000967D187CCB900DDAE0F8A3E0F9A3E0FA91
:10259000A3E0FB120F2E500F900DDAE0FCA3E0FD3C
:1025A000A3E0FEA3E0FF22900DDAE0FCA3E0FDA390
:1025B000E0FEA3E0FF120EAD900DDE12127E900D34
:1025C000DEE0FCA3E0FDA3E0FEA3E0FFEC120E6F53
:1025D000C8ECC8C9EDC9CAEECACBEFCB900DDAE0A2
:1025E000FCA3E0FDA3E0FEA3E0FF120BD4E4FBFAA2
:1025F000F9F8120F2E60264024900DDEE0FCA3E0D7
:10260000FDA3E0FEA3E0FFEF24FFFFEE34FFFEEDAD
:1026100034FFFDEC34FFFC900DDE12127E900DDED7
:10262000E0FCA3E0FDA3E0FEA3E0FFEC120E6F22AE
:100EE400E9D2E7C933E833F892D5EDD2E7CD33EC54
:070EF40033FC5002B2D522CD
:100EFB00EC30E7100FBF000C0EBE00080DBD000458
:100F0B000BEB6014A2D5EB13FCED92E7FD2274FF03
:100F1B00FCFDFEFF22E480F8A2D574FF13FC7D805C
:030F2B00E480EF70
:100F2E0074F8CC6480CCC86480C8F58204604FC36A
:100F3E00EB9FF5F0EA9E42F0E99D42F0E89C45F009
:100F4E00603C501DE5825FFFE582D313CB5BCBF493
:100F5E002B5582FB50280ABA002409B900200880BC
:100F6E001DE5825BFBE582D313CF5FCFF4C3132F56
:100F7E005582FF50090EBE00050DBD00010CC3EBDE
:100F8E009FF5F0EA9E42F0E99D42F0E89C45F06044
:090F9E0007CC4820E701B3EC2266
:03000000022E7B52
:0C2E7B00787FE4F6D8FD758181022EC23C
:100FA700BB010689828A83E0225002E722BBFE0248
:090FB700E32289828A83E493227B
:100FC000BB010CE58229F582E5833AF583E02250E6
:100FD00006E92582F8E622BBFE06E92582F8E22230
:0D0FE000E58229F582E5833AF583E493224A
:100FED00BB010689828A83F0225002F722BBFE01E3
:020FFD00F322DD
:100FFF00F8BB010DE58229F582E5833AF583E8F028
:10100F00225006E92582C8F622BBFE05E92582C8D3
:02101F00F222BB
:10102100C2D5EC30E709B2D5E4C39DFDE49CFCEEEA
:1010310030E715B2D5E4C39FFFE49EFE12136EC3E1
:10104100E49DFDE49CFC800312136E30D507C3E4DC
:061051009FFFE49EFE2259
:10105700C5F0F8A3E028F0C5F0F8E5821582700224
:061067001583E038F022C1
:10106D00A3F8E0C5F025F0F0E58215827002158336
:06107D00E0C838F0E82293
:10108300BB010A89828A83E0F5F0A3E02250068738
:10109300F009E71922BBFE07E3F5F009E3192289FA
:0B10A300828A83E493F5F0740193222D
:1010AE00BB010789828A83021057500B09C5F027AE
:1010BE00F7C5F01937F722BBFE0D09F8E325F0F35B
:1010CE00C5F019E338F322F889828A8374019325D7
:0810DE00F0C5F0F8E49338229C
:1010E600E88FF0A4CC8BF0A42CFCE98EF0A42CFCA9
:1010F6008AF0EDA42CFCEA8EF0A4CDA8F08BF0A427
:101106002DCC3825F0FDE98FF0A42CCD35F0FCEB85
:101116008EF0A4FEA9F0EB8FF0A4CFC5F02ECD394A
:0F112600FEE43CFCEAA42DCE35F0FDE43CFC22B7
:1011350075F008758200EF2FFFEE33FECD33CDCC71
:1011450033CCC58233C5829BED9AEC99E5829840F4
:101155000CF582EE9BFEED9AFDEC99FC0FD5F0D6D1
:10116500E4CEFBE4CDFAE4CCF9A88222B800C1B9FB
:101175000059BA002DEC8BF084CFCECDFCE5F0CB39
:10118500F97818EF2FFFEE33FEED33FDEC33FCEB72
:1011950033FB10D703994004EB99FB0FD8E5E4F92D
:1011A500FA227818EF2FFFEE33FEED33FDEC33FC1A
:1011B500C933C910D7059BE99A4007EC9BFCE99A0E
:1011C500F90FD8E0E4C9FAE4CCFB2275F010EF2F53
:1011D500FFEE33FEED33FDCC33CCC833C810D70753
:1011E5009BEC9AE899400AED9BFDEC9AFCE899F88E
:0E11F5000FD5F0DAE4CDFBE4CCFAE4C8F92221
:0E120300C3E49FFFE49EFEE49DFDE49CFC22FC
:10121100EB9FF5F0EA9E42F0E99D42F0EC6480C854
:0612210064809845F022F4
:10122700EB9FF5F0EA9E42F0E99D42F0E89C45F01D
:011237002294
:10123800E8600FEFC333FFEE33FEED33FDEC33FC14
:03124800D8F122B8
:10124B00BB010789828A8302127E5005E9F80212DC
:0A125B0072BBFE05E9F80213C3227E
:0D126500E6FB08E6F908E6FA08E6CBF822F9
:0C127200ECF608EDF608EEF608EFF622A8
:0C127E00ECF0A3EDF0A3EEF0A3EFF022E3
:10128A00A8828583F0D083D0821212A11212A112F1
:10129A0012A11212A1E473E493A3C583C5F0C58316
:1012AA00C8C582C8F0A3C583C5F0C583C8C582C8AE
:0112BA002211
:1012BB00BB010DE58229F582E5833AF5830213D84C
:1012CB005007E92582F80213CFBBFE07E92582F808
:1012DB000213E1E58229F582E5833AF5830213EAED
:1012EB00D083D082F8E4937012740193700DA3A392
:1012FB0093F8740193F5828883E4737402936860A6
:06130B00EFA3A3A380DFA5
:10131100E5092582F582E5083583F583B50804855D
:1013210082092210AF06858209F50822858209F516
:0413310008D2AF220D
:0D133500E5092582F582E5083583F5832260
:1031F400900DD3EBF0A3EAF0A3E9F0E4900DDBF03B
:10320400A3F0900DD974FFF5F012106D45F0603CF9
:10321400900DD6E0FBA3E0FAA3E0F9120FA7FF900C
:103224000DD3E0FBA3E0FAA3E0F9900DDBE475F025
:103234000112106D85F082F583EF120FFFEF60C26B
:10324400900DD7E475F00112105780B6900DD3E0BD
:08325400FBA3E0FAA3E0F9225C
:10002600900DD6EBF0A3EAF0A3E9F0A3EBF0A3EA78
:10003600F0A3E9F0900DD9E0FBA3E0FAA3E0F912F2
:100046000FA7600C900DDAE475F00112105780E4EA
:10005600900DD9E0FBA3E0FAA3E0F9120FA76D70AB
:100066000122900DD6E0FBA3E0FAA3E0F9EBC0E095
:10007600EAC0E0E9C0E0A3E0FBA374FFF5F01210CC
:100086006DFAD082D083D0E06B7009E5F06582709E
:0A00960003EA658370BAFBFAF92251
:10134200EF4E6012EF60010EEDBB010B89828A83C2
:10135200F0A3DFFCDEFA2289F05007F709DFFCA9CF
:0C136200F022BBFEFCF309DFFCA9F02226
:102E87000237A1E493A3F8E493A34003F68001F289
:102E970008DFF48029E493A3F85407240CC8C3334C
:102EA700C4540F4420C8834004F456800146F6DF1B
:102EB700E4800B01020408102040809037F9E47E7B
:102EC700019360BCA3FF543F30E509541FFEE49310
:102ED700A360010ECF54C025E060A840B8E493A3D7
:102EE700FAE493A3F8E493A3C8C582C8CAC583CA02
:102EF700F0A3C8C582C8CAC583CADFE9DEE780BEBA
:0138220000A5
:10136E00BC000BBE0029EF8DF084FFADF022E4CC63
:10137E00F875F008EF2FFFEE33FEEC33FCEE9DEC2C
:10138E00984005FCEE9DFE0FD5F0E9E4CEFD22ED72
:10139E00F8F5F0EE8420D21CFEADF075F008EF2FBC
:1013AE00FFED33FD4007985006D5F0F222C398FDAD
:0513BE000FD5F0EA224A
:0C13C300ECF208EDF208EEF208EFF22266
:0913CF00E6FB08E6FA08E6F92243
:0913D800E0FBA3E0FAA3E0F92216
:0913E100E2FB08E2FA08E2F9223D
:0C13EA00E493FB740193FA740293F9225F
:00000001FF
